:020000040800F2
:100000000020002075230008192000081B2000088C
:1000100000000000000000000000000000000000E0
:100020000000000000000000000000001D2000088B
:1000300000000000000000001F2000082120000830
:10004000C523000800000000C5230008C5230008E0
:10005000C5230008C52300082D200008372000080C
:10006000000000004120000851200008C5230008BE
:10007000C5230008C5230008C523000800000000B0
:10008000C52300080000000000000000C523000890
:1000900000000000C5230008C5230008C523000890
:1000A000C5230008C5230008C523000869200008EF
:0800B000C52300080000000058
:1000B80010B5064C2378002B07D1054B002B02D036
:1000C800044800E000BF0123237010BD6400002035
:1000D800000000009C640008044B10B5002B03D0FE
:1000E8000349044800E000BF10BDC04600000000FE
:1000F800680000209C6400080023C25C0133002AC9
:10010800FBD1581E7047000002B4714649084900E7
:10011800095C49008E4402BC7047C046002243086F
:100128008B4274D303098B425FD3030A8B4244D3B7
:10013800030B8B4228D3030C8B420DD3FF220902F9
:1001480012BA030C8B4202D31212090265D0030BB8
:100158008B4219D300E0090AC30B8B4201D3CB03AE
:10016800C01A5241830B8B4201D38B03C01A5241F0
:10017800430B8B4201D34B03C01A5241030B8B42F2
:1001880001D30B03C01A5241C30A8B4201D3CB02DD
:10019800C01A5241830A8B4201D38B02C01A5241C2
:1001A800430A8B4201D34B02C01A5241030A8B42C5
:1001B80001D30B02C01A5241CDD2C3098B4201D3DD
:1001C800CB01C01A524183098B4201D38B01C01A5B
:1001D800524143098B4201D34B01C01A52410309D2
:1001E8008B4201D30B01C01A5241C3088B4201D381
:1001F800CB00C01A524183088B4201D38B00C01A2E
:10020800524143088B4201D34B00C01A5241411A54
:1002180000D20146524110467047FFE701B5002061
:1002280000F0F0F802BDC0460029F7D076E7704725
:1002380003460B437FD4002243088B4274D303093F
:100248008B425FD3030A8B4244D3030B8B4228D3E0
:10025800030C8B420DD3FF22090212BA030C8B4206
:1002680002D31212090265D0030B8B4219D300E0A6
:10027800090AC30B8B4201D3CB03C01A5241830B2B
:100288008B4201D38B03C01A5241430B8B4201D3DB
:100298004B03C01A5241030B8B4201D30B03C01A04
:1002A8005241C30A8B4201D3CB02C01A5241830A7E
:1002B8008B4201D38B02C01A5241430A8B4201D3AD
:1002C8004B02C01A5241030A8B4201D30B02C01AD7
:1002D8005241CDD2C3098B4201D3CB01C01A52413E
:1002E80083098B4201D38B01C01A524143098B42C7
:1002F80001D34B01C01A524103098B4201D30B01B0
:10030800C01A5241C3088B4201D3CB00C01A5241D4
:1003180083088B4201D38B00C01A524143088B4299
:1003280001D34B00C01A5241411A00D20146524132
:10033800104670475DE0CA0F00D04942031000D351
:100348004042534000229C4603098B422DD3030AA6
:100358008B4212D3FC22890112BA030A8B420CD3B6
:10036800890192118B4208D3890192118B4204D3DF
:1003780089013AD0921100E08909C3098B4201D35F
:10038800CB01C01A524183098B4201D38B01C01A99
:10039800524143098B4201D34B01C01A5241030910
:1003A8008B4201D30B01C01A5241C3088B4201D3BF
:1003B800CB00C01A524183088B4201D38B00C01A6C
:1003C8005241D9D243088B4201D34B00C01A524143
:1003D800411A00D20146634652415B10104601D3D0
:1003E8004042002B00D54942704763465B1000D35A
:1003F800404201B5002000F005F802BD0029F8D000
:1004080016E770477047C0468446100062468C461F
:100418001900634600E0C0461FB500F0ABFF002896
:1004280001D40021C8421FBD10B500F0EBFE4042C8
:10043800013010BD10B500F09DFF002801DB002041
:1004480010BD012010BDC04610B500F093FF002874
:1004580001DD002010BD012010BDC04610B500F020
:1004680015FF002801DC002010BD012010BDC0468A
:1004780010B500F00BFF002801DA002010BD0120A4
:1004880010BDC0469E2110B5C905041C01F00AFB29
:10049800002803D1201C00F0EFFA10BD9E21201C7B
:1004A800C90500F045F900F0E7FA80231B069C46D1
:1004B8006044F2E7F0B54F464646D64643025B0A2B
:1004C8004500C0B599460F1C2D0EC60F002D00D152
:1004D80088E0FF2D00D18DE08022DB00D2041A4392
:1004E8000023914698469A467F3D7C027B00640A29
:1004F8001B0EFF0F002B68D0FF2B21D08022E400B9
:10050800D204144342467F3B5B1900215D1C0A2A32
:100518002EDC7E404246022A23DC013A012A00D919
:10052800BDE002296ED001292CD100200022C0058F
:10053800F60710433043E0BCBA46B146A846F0BDC2
:100548002B00FF33002C65D00322414611433200B3
:10055800013588467A40FF350A2900DDD8E01600C3
:100568000321404601228240A620C000024220D03A
:100578005346022B46D0032B00D1BBE051464C46D4
:100588000129D2D02B007F33002B70DD620704D005
:100598000F222240042A00D00434220103D5634BE1
:1005A8001C402B008033FE2B2CDCA201520AD8B24F
:1005B800BDE790208000024227D1B938FF381042A9
:1005C8006DD03E00A1468A46D2E7002C41D10123D6
:1005D80042461A4390462B00424601215D1C0A2AD6
:1005E80097DDC5E7002B26D104239846033B002559
:1005F8009A467AE7002B18D108239846063BFF2530
:100608009A4672E7FF20002291E780220026FF2009
:10061800D2038CE741460222013511438846FF3553
:100628000A29A5DC02217E4074E70C239846093B81
:10063800FF259A4659E7180001F03EFA4A46431F3B
:1006480076259A4000236D42914698469A462D1A7F
:100658004BE7200001F030FA4246431F9C402B1A1A
:10066800763B00215D1C0A2A00DC52E780E7012264
:10067800D31A1B2B00DD58E79E352200AC40DA4028
:10068800631E9C412243530704D00F231340042BBD
:1006980000D00432530137D50120002247E7210C4E
:1006A8004A462404240C2700100C1204120C44435C
:1006B8005743484351433A0C09195218944203D9F5
:1006C800802149028C4660443F0411043F0CC9193B
:1006D8008C01671EBC41120C890E12180C43920142
:1006E800144312010ED5012362081C40144349E744
:1006F8003E00A14680224B46D2031A435202FF20F5
:10070800520A14E71D003DE792010020520A0EE745
:100718000F29EDD180224B46D2031342EAD014426E
:10072800E8D13E00FF20224301E7C046FFFFFFF764
:10073800F8B54746CE464E0243024500720AC40F3A
:10074800480080B594465F0A2D0E9B09000EC90F1C
:10075800B609FF2824D0012251402A1A8C420FD012
:10076800002A00DC6AE1002835D1002E00D1A2E081
:10077800511E012A00D124E1FF2A21D00A002FE0CE
:10078800002A00DC67E100285ED0FF2D18D0802108
:10079800C9040E431B2A00DC76E02A00013332E04C
:1007A8002A00FF3A9146002E42D08C4255D04A4644
:1007B800002A00D19CE0002D00D177E00C00330026
:1007C800DB08002B00D16EE08022D20313435B02CA
:1007D800FF205B0A24E0FF2DF2D08021C9040E43DC
:1007E80001211B2A08DC31002020D140821A9640C2
:1007F8003200501E824111435B1A5A0160D407210E
:100808002A00194057D00F211940042900D0043379
:10081800590150D5501CFE2A45D09B01C0B25B0A35
:10082800C0051843E4072043C0BCB946B046F8BD2C
:10083800012251408C42BAD14A46002A10D0002DDC
:1008480000D198E00023BBE7002E34D0511E012AC6
:100858006ED0FF2AB4D00A009CE7002A00D088E0B6
:10086800FE206A1C104200D092E0002D00D0A4E0C7
:10087800002B00D1CBE0002E00D0CAE00022DB081C
:100888005B025B0AD0B2CBE731002020D140821A4C
:1008980096403200501E82410A439B185A01AED539
:1008A8006A1CFE2D4AD1FF200023B9E7FF22002B46
:1008B8004BD10C003300DB08FF2A00D181E7DFE7CA
:1008C8009F01BF09380001F0F7F8053887408542D5
:1008D80021DC3B002021421B0132D3408A1A974079
:1008E8007A1E974100223B43590700D08BE78FE7D8
:1008F800FE206A1C104212D1002D52D1002B7CD050
:10090800002EBBD09A1B500100D48BE0012400229A
:10091800F31A0C40E8E7564B2A1A3B40E4E79F1BC2
:100928007A0146D4002FCDD100240020002377E798
:100938009B1901250132590100D460E701214D4876
:1009480019405B0803400B43CEE7571E012A5AD0D3
:100958000C00FF2A33D001221B2F07DC2021C91BE2
:100968001A008B40FA40591E8B411A430500B31AEE
:1009780043E7002D23D1FF22002B9BD0511E012AD3
:10098800D6D0FF2A1BD01B292CDD0200731C3AE7A6
:10099800FF2A88D09B195B08590700D033E7DB088A
:1009A8006EE7002B10D1002E43D0012433000C40F9
:1009B80006E70124F71A0C4084E7002B04D1330022
:1009C800FEE601259B1B18E7002E00D1F8E68022E1
:1009D800D203974204D3944502D2012433000C4039
:1009E800DB08F1E61A002025CA40691A8B40591E17
:1009F8008B41134305009B1950E7002E94D0012426
:100A080033000C403AE70C000125F31AF5E63300F1
:100A180034E79B1900225901C1D5154A1340DB0858
:100A280001222DE7002A00D17EE713000022DB080F
:100A380026E780230024FF20DB03F1E6002A00D10B
:100A480056E7471B3A00002D00D130E78022D20438
:100A58000C0013437FE7002A00D101E7411B002D5A
:100A680001D10A0088E78022D20413438BE7C046ED
:100A7800FFFFFFFBFFFFFF7D41024200C30F490A52
:100A88000020120E7E2A03DD9D2A02DD094A9818ED
:100A98007047802000040143952A07DC9620821ABB
:100AA800D1404842002BF3D10800F1E7963A914033
:100AB800F7E7C046FFFFFF7F70B5041E0ED000F0B9
:100AC800FBFF9E2301001B1A962B0CDC08282FD055
:100AD80008398C406402640AD8B201E0002000247E
:100AE800C005204370BD992B16DC421F052800D095
:100AF8009440220010480240650709D00F252C4079
:100B0800042C05D00432540102D59F2302405B1AFD
:100B18009201540AD8B2E3E7020020001B32904049
:100B28000200501E82410520401AC4401443E0E7E9
:100B380064029620640AD3E7FFFFFFFBF0B557462F
:100B48004E464546DE46E0B583B0009001910C0361
:100B58004F00CE0F610A009C1D03640F0C430099DF
:100B680000920193C80059004B0D9946009A019BC9
:100B78006D0AD90F530F2B439A46009B7F0DDA005D
:100B880094464A46B046BA1A8E4200D1B0E0002ACE
:100B980000DC78E04946002900D1E9E0C9498F42E4
:100BA80000D195E10125382A16DC80215346090435
:100BB8000B439A461F2A00DDE7E1202155468B1A90
:100BC80061469D40D1400D43614699404B1E994175
:100BD8005346D3400D43E41A451BA8428041404286
:100BE800241A230200D40FE16402640A002C00D105
:100BF80039E1200000F060FF0300083B20212800B5
:100C0800CA1AD0409C4002009D4022439F4200DD0A
:100C180073E1D81B0130091A2C008D40C4406B1EAB
:100C28009D411300C2408B402543002714001D43FB
:100C38006B0709D00F232B40042B05D02B1DAB428B
:100C4800AD416D4264191D00230200D42DE19D4A77
:100C58000137974200D1D3E046469B49ED08214031
:100C68004A072A437C054D022D0B640D24052C43AD
:100C7800F60734431000210003B0F0BCBB46B2466F
:100C8800A946A046F0BD002A00D184E04A46D21BFE
:100C9800002F00D06DE12500054300D127E1561E45
:100CA800012A00D13BE2874DAA4200D16AE2012520
:100CB800382E12DC32001F2A00DDF8E1202625003C
:100CC800B61A07005346B040D440B540D740461E38
:100CD800B0411B1B9A463D4305436246551BAC4534
:100CE8009241534652420E004F4688469C1A78E776
:100CF800002A00DC8EE04946002975D1614653463A
:100D0800194300D1F6E0511E012A00D191E16D4D41
:100D1800AA4200D1DCE00125382914DC0A001F2A88
:100D280000DDA2E120215346891A8B401D0063464D
:100D3800D3401D4363468B4019004B1E99415346CF
:100D4800D3400D43E4182D188542804140422418B1
:100D5800230259D55B4B01379F4251D001215A4B91
:100D68006A081C4029400A43E507154364085FE701
:100D780061465346194300D1BCE0511E012A00D1F7
:100D880064E1504DAA4200D16AE10125382900DD0D
:100D980022E70A000EE74D4A7D1C154200D0D0E03C
:100DA80025006246534605431A43002F00D037E119
:100DB800002D00D1A8E1002A00D16AE16346C51AD6
:100DC8005346E21AA8429B415B42D31A1A0200D446
:100DD80003E263461D1AAC459241534652421C1B1E
:100DE8000E008846A41A23E736498F4270D00125A1
:100DF800382AA8DC8021534609040B439A468EE71B
:100E08003C000025002231E707232B40002B00D0AF
:100E180010E793E0002A74D04A46D21B002F00D175
:100E2800C7E02849894500D185E10125382A12DC27
:100E3800802109040C431F2A00DDABE12021250095
:100E4800891A070088408D40D740411E8841D44008
:100E58003D430543A244654465459241524252448C
:100E680014004F4674E7280000F026FE03001833EC
:100E78001F2B00DCC2E62A00083882409F4200DDB2
:100E8800A9E0DB1B581C1F2800DCACE115001F3B48
:100E9800DD40202805D040231B1A9A40531E9A4152
:100EA8001543072300272B40B0E7ED08054B6207E1
:100EB8002A43E4089F420FD02403250B7C05640DC8
:100EC800D4E6C046FF070000FFFF7FFFFE070000D3
:100ED800C00862070243E4081300234300D186E1F7
:100EE80080252D0325432D03C34C2D0BBEE66046FC
:100EF80054460E001700C508D8E7C04CFF1A144026
:100F080096E6BF4A791C11426BD122000243002F9A
:100F180000D0DBE0002A00D12DE1624653461A4397
:100F280000D1B6E06346C51885428041544440422A
:100F38002418230202D50F00B04B1C403A002800A9
:100F4800D8E76246851AA8429241534652429146D2
:100F5800E31A1A004B46D21A130091461A0254D4C7
:100F68004A464C462A4300D040E600260024002585
:100F78007CE6A14DA94500D190E00125382A00DD85
:100F8800ABE680252D042C4395E611005546203903
:100F9800CD40A946202A06D0402153468A1A9340BC
:100FA80062461A43944665466B1E9D414B461D4357
:100FB80012E62100014300D1C4E0511E012A00D1EC
:100FC800FBE08D4DAA4200D1B5E00125382900DDAE
:100FD80041E70A002FE7894CFF1A14406207E4082A
:100FE8006AE7854A914200D1E3E06346C21882422B
:100FF80080412300404253441B18DD075C08072347
:10100800520815430F002B4000E763461D1AAC45F4
:101018009241534652421C1B0E008846A41AE5E52D
:10102800002D00D091E0002A38D180240026240326
:1010380056E76346C5188542804154444042241807
:101048000127230200D4DFE6022787E66346C51A94
:10105800A842804153464042E41A0127241AC0E5B9
:101068006207C0080243E40836E7110053462039F6
:10107800CB409946202A06D0402153468A1A9340ED
:1010880062461A43944665466B1E9D414B461D4376
:1010980059E66207C0080243E4080DE753465A07B9
:1010A8006346D80853460E000243DC0814E71500CF
:1010B8002600203DEE40202A03D04025AA1A94405D
:1010C8002043421E90410500354306E6002A7CD0A5
:1010D80062465346C0081A4300D1FAE66207104335
:1010E8008022E4081203144208D0D908114205D11D
:1010F8006346D80853460C005B071843420FC000EC
:10110800C00852070243E7E6002A00D12DE76346EC
:10111800D80853465A070E000243DC08CCE663465B
:101128001D1AAC459241534652421C1B0E0088467C
:10113800A41A013755E56346D90853465A070A43A6
:10114800DC08C9E660465446D4E6C008002A00D147
:10115800BFE6620710438022E40812031442CDD090
:10116800DD081542CAD16346D80853465B070E000E
:101178002C001843C2E76346D90853465A070A4366
:10118800DC0899E66346D80853465A070E0002431E
:10119800DC08A1E6110027002039CF40202A03D01F
:1011A80040218A1A94402043421E904105003D4345
:1011B80051E60C000025002258E560446045924144
:1011C800544452420500A4183AE753465A07634666
:1011D800D90853460A43DC087EE61A001C002A4355
:1011E80000D0ABE6C1E620210025091A19E5002246
:1011F8000025014C3AE5C046FF070000FFFF7FFFCE
:10120800FE070000F0B55746DE464E464546E0B5B7
:101218000D000400E80F83460903D80F090B824626
:1012280019488C461F0369005E00490D3F0B760D77
:10123800814218D086420FD00120B1420DD1BC4561
:101248000BD1944209D1D3451CD0002905D1604661
:101258002043431E984100E00120F0BCBB46B24643
:10126800A946A046F0BD01208E42F6D16146394319
:101278000F0017432743F0D15B465246981A431E86
:101288009841EAE70020E8E7FF070000F0B5574675
:101298004E464546DE46E0B50D000F03390B83B0D8
:1012A8000400804601915800E90F314F400D8C46EB
:1012B8006E00190382469146760D090BD80FBE427F
:1012C8001FD0BA450FD0002E2FD15546019E34436A
:1012D800002D27D10A433AD0002C45D100281AD135
:1012E8000120404217E011433BD1002E02D1019F5B
:1012F8002743F3D0844509D16346002BF0D06046DC
:1013080009E0019F27432CD1B24524D0634602202F
:10131800013B1840013803B0F0BCBB46B246A946B1
:10132800A046F0BD002CD9D0E4E75446002CEDD0FF
:101338008445EBD15645E9DCDEDB019B8B42E5D8E1
:10134800DAD1C845E2D80020C845E4D2D4E7002065
:10135800002CE0D0DAE7114303D18445D6D1002030
:10136800D9E702204042D6E78445E6D0CEE7C0461A
:10137800FF070000F0B557464E464546DE46E0B545
:101388000D000F0304008046E80F390B844683B034
:101398005800304F400D01911E0369008246914666
:1013A800490D360BD80FB94220D0BA450FD00029C5
:1013B8002BD101990C435146002937D1324338D0FB
:1013C800002C44D1002819D10120404216E01643D0
:1013D80013D1002902D1019F2743F3D0844520D09F
:1013E80063460220013B1840013807E0019F27436C
:1013F80003D18A45F4D116431FD0022003B0F0BCB4
:10140800BB46B246A946A046F0BD5446002CE7D0DC
:101418008445E5D15145E3DC03DB019BB342DFD8CA
:101428000FD06346002BCFD06046E7E7002CC9D029
:10143800D4E70020002CE1D0D2E78445D0D10020A9
:10144800DCE7C845CCD80020C845D7D2E9E78445B1
:10145800E3D0C5E7FF070000F0B55746DE464E4625
:101468004546E0B51F000B031B0B16009A46CA0F32
:101478004B000400934687B05B0D00D1D5E0BB4A12
:10148800934200D1F8E05146420FC9000A43802137
:1014980009041143C2009146B54A8A469D180023A3
:1014A800984602933C037B00FA0F3000240B5B0D37
:1014B800009200D196E0AD4A934231D0720FE40019
:1014C8002243802424041443A94AF0009446634428
:1014D8005B195A1C0192424600260A2A42DC5A46E7
:1014E80000994A4093464246022A32DC013A012AD0
:1014F80000D949E1022E00D1CAE0012E3DD10023D6
:101508000024002210005A461B052343D207134328
:10151800190007B0F0BCBB46B246A946A046F0BDCC
:10152800924B2643EB18002E00D1BBE00322414624
:1015380011435A46884600994A40802109018C4641
:1015480029006144019141460A2900DD33E29346AE
:101558000326424601279740A6213A00C9000A40BF
:101568000F4231D0029E022E00D135E2032E00D167
:10157800D2E154464846012EC1D0019A7D4B94468B
:101588006344002B00DCC0E0420709D00F22024070
:10159800042A05D0021D82428041404224181000CE
:1015A800E20106D5744B019A1C4080239446DB0067
:1015B8006344724A93426BDC6207C00864025B05AD
:1015C8000243240B5B0D9DE7902189000F4263D1F4
:1015D80088223A4200D1D7E0009BA2469B4681462A
:1015E8000296BFE72300334300D17FE0002C00D1EF
:1015F800ADE1200000F060FA020003000B3A1D2064
:101608001900821A30000839D0408C400443300059
:1016180088405B4AEB1A944663445A1C019242463E
:1016280000260A2A00DC5AE79CE7534603439946FA
:1016380054D05346002B00D177E1504600F03CFAD5
:101648000B235B429C460200844411005046083933
:1016580088401D23804660461B1A2000D84003009E
:10166800404603439A4623008B4099460023444D45
:101678009846AD1A029315E752460243914626D181
:1016880000221D000223924608329046029309E781
:1016980000240022354B35E7002380249B46240391
:1016A800324B2FE702224146114380221201944611
:1016B8002A006244884601920A2900DD52E75A4608
:1016C8000020009904004A40934602260BE70C22AA
:1016D8001D000323814690460293E3E600239A46C1
:1016E80004339846033B00250293DBE64246013368
:1016F8001A432B0090465A1C0192424600240020AF
:1017080001260A2A00DCEAE62CE70122D21A382A46
:1017180000DDF4E61F2A00DC2AE11F214942CB1A2A
:101728002100D9400B00202A05D0164A019D944675
:101738006544AC402043421E9041184307231900DA
:101748000024014003420CD00F230340042B00D196
:1017580040E1031D8342A44118006442610764020A
:10176800240BC20800230A43CCE6C046FF0700004A
:1017780001FCFFFFFF030000FFFFFFFEFE07000064
:101788000DFCFFFF3E04000049464A460904090CC7
:101798000D00160C020C0004000C4543AC46050075
:1017A8007543A84615000F007543009202952A005C
:1017B800009D6F4365462D0CA94647444F44B845E4
:1017C80005D91500802252029046454402953D0CE9
:1017D800039565462D043F042D0CAC463D00654439
:1017E8000495250C2404240CAC4625007543A84612
:1017F80065460F006943414489466743390C4944AB
:101808006E43884503D980225202904646440D0C07
:10181800A846350045440595039D3F04A8463F0C5E
:101828000904C91988444546039555462E04360CC3
:101838002F0C35004543784381463800A8462D0CC7
:10184800AA46009A504372434A445244914503D9E8
:1018580080256D02A9464844150CA94645462D0425
:101868002D0CA84665467D43120448449044A94679
:101878003200654662436E437C43170C3619BF1924
:10188800BC4203D980246402A446E144029C039E1E
:10189800A446059D66448E428941AC4612043C0428
:1018A800120CA2186244494254184644A4464645BC
:1018B800A44182466442A046AA4292418C4589418D
:1018C800E244D044494252420A43A045A4418245D9
:1018D8008941644249420C4341463F0CD2191219CE
:1018E800CC0D049970020843411E884141464A4480
:1018F800F60D52023043490214430843D20135D54C
:101908000122430802401343E0071843640834E601
:10191800009BA2469B4681468024534624031C43D1
:1019280024034A462E4B240BECE500F0C5F815239A
:101938009C4684440200634620321C2B00DC84E66B
:10194800002399462300083883409A468EE600F023
:10195800B3F802000300153220331C2A00DC4EE6DF
:1019680002003400083A0020944052E6019304E64D
:101978001C4B21009C460300019DD3406544A940AF
:1019880019430300AB40581E834119430800D44053
:101998004B0709D00F230B40042B05D00B1D8B429E
:1019A8008041404224181800230200D4D6E60123BF
:1019B80000240022A6E50F29AAD1802352461B0342
:1019C8001A42A9D01C42A7D11C43009B02009B4687
:1019D800034B97E50024C1E60024014B220091E562
:1019E800FF0700001E04000070B5002816D0C317BA
:1019F800C5185D40C40F280000F05EF8104B1B1A94
:101A08005B055B0D0A2814DC02002E001532964097
:101A18000B22121AD5402D032D0B03E000240023BE
:101A2800002500261B052B43E4072343300019003B
:101A380070BD0B3885402D0300262D0BF2E7C046FC
:101A48001E040000844608006146FFE71FB500F049
:101A5800C9F8002801D40021C8421FBD10B500F004
:101A680049F84042013010BD10B500F0BBF800281D
:101A780001DB002010BD012010BDC04610B500F0EC
:101A8800B1F8002801DD002010BD012010BDC046BE
:101A980010B500F057F8002801DC002010BD012027
:101AA80010BDC04610B500F04DF8002801DA00203E
:101AB80010BD012010BDC0461C2101231B04984203
:101AC80001D3000C10391B0A984201D3000A0839C7
:101AD8001B09984201D30009043902A2105C40187E
:101AE8007047C04604030202010101010000000022
:101AF8000000000070B542004E024C0045026D0A1D
:101B0800120EC30F760A240EC90FFF2A10D0FF2C1D
:101B18000CD00120A2420AD1B54208D18B420FD085
:101B2800002A04D12800431E984100E0012070BD1E
:101B38000120FF2CFBD13543F9D14B401800F6E7C3
:101B48000020F4E730B5420044024D02C30F4800BC
:101B5800640A120E6D0A000EC90FFF2A19D0FF2859
:101B68000BD0002A1ED100280BD1002D27D0002C25
:101B780034D100292FD0080030BD002D28D1002AEB
:101B880001D1002CF5D08B4207D1002B23D01800AF
:101B9800F2E7002C1CD1FF2814D0581E022318404D
:101BA8000138E9E70028F8D08B42F6D18242F4DC0C
:101BB800EBDBAC42F1D80020AC42DDD2E5E7002CEB
:101BC800DAD0EAE7002D03D18B42E6D10020D3E733
:101BD80002204042D0E701204042CDE78B42E8D0C6
:101BE800DBE7C04630B5420044024D02C30F48004F
:101BF800640A120E6D0A000EC90FFF2A1AD0FF28B8
:101C08000ED0002A1ED100280ED1002D2AD0002C7B
:101C18000CD08B421DD0581E02231840013810E00A
:101C2800002D0DD1002A20D1002C1ED1002923D04F
:101C3800080006E0002C03D1FF28ECD1002D17D0B6
:101C4800022030BD0028E6D08B42E4D18242E2DC9B
:101C580004DBAC42DFD80020AC42F2D2002B0BD020
:101C68001800EEE7002CECD0D5E78B42D3D1F5E78E
:101C780000208B42E5D0CEE701204042E1E7C04694
:101C88001FB50C22002101A804F0CEFB8022184CBD
:101C9800184B120622610422236080236261033AF2
:101CA8001B03A276E2612200636000232C321370CA
:101CB80007226263220020003C32A360E360238392
:101CC8006362A36223631370E36400F0CBFB002814
:101CD80001D000F083F9084B20000193012301A9EA
:101CE800029300F027FD002801D000F077F91FBD0E
:101CF800DC000020002401400200000470B505004B
:101D08008EB01422002103A804F08EFB18220021B3
:101D180008A804F089FB264B2A689A4245D18023FB
:101D2800DB010893802308A81B060C9301F078FFB9
:101D3800002801D000F052F980211E4B49031A6C8B
:101D4800A0200A431A641A6C00260A400121019255
:101D5800019A5A6BC0050A435A635B6B05960B40A0
:101D68000293029B022303935B1803A9049301F0D7
:101D780083FA114C114B20002360052363607B33E9
:101D88002361803363618023DB00A3612023E36147
:101D980080235B01A660E660236200F0D9FFB042B1
:101DA80001D000F01BF92C65A5620EB070BDC046CD
:101DB800002401400010024080000020080002407A
:101DC80007B501210C4B09209A6B0A439A639B6B58
:101DD80000220B4001934918019B00F01FFF0920C6
:101DE80000F046FF002202210A2000F017FF0A2017
:101DF80000F03EFF07BDC04600100240F0B50227C4
:101E08000125A02689B01422002103A804F00CFBA8
:101E1800394BF6055A6B30003A435A635A6B3749C7
:101E28003A400192019A5A6B00242A435A635B6B29
:101E38002A002B400293029B01F048FB300000224D
:101E4800202101F043FB2A0029002D4801F03EFB28
:101E58000423300003A9039304950594069401F024
:101E68000BFA08230393C42330009B0303A90493AC
:101E7800059401F001FA2023300003A90393049587
:101E88000594069701F0F8F94023300003A903935D
:101E98000494059401F0F0F980230393882330001B
:101EA8005B0303A90493059401F0E6F903A9144818
:101EB800039504950594069401F0DEF9C0235B01AF
:101EC80003931123300003A904930594069701F0A6
:101ED800D3F922003900062000F0A0FE062000F009
:101EE800C7FE22003900072000F098FE072000F006
:101EF800BFFE09B0F0BDC046001002400418000043
:101F0800000400500848094B10B5036003234360E0
:101F1800074BC360074B836001F0FAFA002801D031
:101F280000F05CF810BDC0464001002000300040C1
:101F3800FF0F0000B80B000010B592B0342200214A
:101F480005A804F071FA1022002101A804F06CFA27
:101F58008020800001F016FB0A230593F6330893CE
:101F6800002309930E9308330F9380239B0240228A
:101F78001093802302240A929B053F3A05A80B92EE
:101F88000C940D94119301F029FB002801D072B62E
:101F9800FEE7072303900490210001A8019302940F
:101FA80001F07CFD002801D072B6FEE712B010BD2A
:101FB80010B500F02DFAFFF7BFFF04F047F9FFF75F
:101FC8001DFFFFF7FDFEFFF75BFE00F0B9F800F01C
:101FD800F3F8FFF797FF03F07FFFFEE772B6FEE71F
:101FE80001210A4B82B01A6C0A431A641A6C0A401F
:101FF80080210092009ADA6B49050A43DA63DB6BA9
:102008000B400193019B02B07047C046001002408C
:10201800FEE7FEE77047704710B500F00DFA04F0D0
:1020280047F910BD10B5082001F05EFA10BD10B5D3
:10203800802001F059FA10BD10B5024800F0E2FF07
:1020480010BDC0468000002010B5034800F0DAFF3C
:10205800024800F0D7FF10BDF80100209C010020C5
:1020680070B5134C200002F03BFB200002F07CFA14
:10207800102223680F4DD969114212D01A620E4AF4
:102088001378002B0DD10D4B0D481B685968802320
:102098005B425B1ADBB2137012782900D2B204F0EB
:1020A800EFF929008022200002F05AFF70BDC046D7
:1020B8005402002073060020F3060020F8010020D7
:1020C8007305002070470000084B026882B09A42EE
:1020D80009D18021064B09021A6C0A431A641B6C49
:1020E8000B400193019B02B07047C046002000409E
:1020F8000010024010B5040086B01422002101A887
:1021080004F092F90C4B22689A4213D101210B4B2F
:10211800A0205A6BC0050A435A635B6B0B400093BF
:10212800009B102301930E3B029301A902330593F0
:1021380001F0A2F806B010BD0020004000100240D7
:1021480010B588B01C22002101A804F06DF9174CC5
:10215800174B184A23600223636000232000A36002
:10216800E2602361A36101F08BFF002801D0FFF733
:1021780035FF200001F0AEFF002801D0FFF72EFF49
:1021880060230193FA2300229B00200001A90293F7
:102198000392059202F004F8002801D0FFF71EFF11
:1021A8002000FFF7A7FF08B010BDC046500100206F
:1021B80000200040E703000010B5184B184C0C2213
:1021C800236096239B01636000232000A360E360E3
:1021D80023616261A361E36123626362A36202F027
:1021E80035FE002801D0FFF7F9FE0021200002F09B
:1021F8002FFF002801D0FFF7F1FE0021200002F098
:1022080047FF002801D0FFF7E9FE200002F002FF97
:10221800002801D0FFF7E2FE10BDC046003801409B
:102228005402002070B506008EB01422002103A8C5
:1022380004F0FAF81822002108A804F0F5F8334B46
:1022480032689A4260D1012308A8089301F0E8FC9B
:10225800002801D0FFF7C2FE80212D4BC9011A6C5E
:1022680000250A431A641A6C2A480A400192019A06
:102278000222596B114359635B6B03A91340029304
:10228800029BC0230492039305950695079500F0D9
:10229800F3FF214C214B20002360322363604E332F
:1022A800236180235B01A560E5606561A561E56147
:1022B800236200F04DFDA84201D0FFF78FFE331DC9
:1022C800DC67A662164B174C8022236033236360B9
:1022D800233BA3600023E3606361A361E361802380
:1022E80020005B012261236200F032FD002801D04A
:1022F800FFF774FE1B2000220121F467A66200F09C
:102308008DFC1B2000F0B4FC0EB070BD00380140FD
:102318000010024000040050F80100201C00024098
:10232800300002409C0100200C4B026810B50400EC
:102338009A4212D10A4A0B49136C0B480B4013649A
:10234800C02101F04BF8231DD86F00F05BFDE06F52
:1023580000F058FD1B2000F097FC10BD003801402C
:1023680000100240FFBFFFFF000400500D488546E3
:10237800FFF7A8FE0C480D490D4A002302E0D45887
:10238800C4500433C4188C42F9D30A4A0A4C0023B7
:1023980001E013600432A242FBD304F04DF8FFF7CA
:1023A80007FEFEE700200020000000206400002057
:1023B8005C650008640000204C070020FEE7000070
:1023C80070B5104B05001978002901D1012070BDA6
:1023D800FA208000FDF7A2FE0B4C01002068FDF7F3
:1023E8009DFE00F061FC041EF0D1032DEED8020022
:1023F80001202900404200F011FC044B20001D6020
:10240800E5E7C04604000020000000200800002086
:102418008023084A5B00116810B50B430320136042
:10242800FFF7CEFF041E03D1FFF7DAFD200010BD31
:102438000124FBE700200240034A044B11681B7883
:102448005B1813607047C046E802002004000020B3
:10245800014B18687047C046E802002080684007B2
:10246800C00F70470023F0B585B00400039398426D
:1024780000D1F0E0856D9D4205D1FFF73FFC2300B8
:102488005433E5651D70802325685B05AA681A42E8
:1024980000D1A7E00022AB680192DB0008D410232A
:1024A8000126A26D01961343A365E36D3343E365EB
:1024B8002800FFF7D3FF1022A36D1340034300D079
:1024C800CCE0A26D674B20691A400633FF331343F3
:1024D800A365AB68DB0761D4276BE1687B1E9F416E
:1024E800A368A27E0B43217E3F0389030B43617ED1
:1024F800C9030B4351030B439C46002800DB86E0CD
:1025080041004908230066462C331B785B0033439F
:102518003B430B43611CC97F012905D1002A00D028
:1025280078E0802252021343626A002A05D0E02133
:1025380049000A40A16A0A431343EA684A490A4023
:102548001343EB60230062683C33E16C1B78970F00
:10255800BF079C463943012B08D1236C666C334373
:102568000B43A16C0B4361463B4319432B693F4F17
:102578003B400B4380212B6153005B08C9058B420C
:102588000CD080231B069A4208D03949394F0B6872
:102598003B40F027BF033A4013430B6007217027E5
:1025A8006B69626B8B4313436B616969A36BB943B6
:1025B8001B010B436B61002834D11023A96A5B42CD
:1025C8000B43AB6207216B690B409A4239D1002358
:1025D800E365A26D03339A43023B1343A365019855
:1025E80005B0F0BDAA6824490A401343AB60234BE9
:1025F80023491868FDF792FD013040000390039BC2
:10260800002B00D146E7039B013B0393F7E78021AA
:10261800890377E72022A76D3A43A265E26D11434B
:10262800E16581E780239B039842CBD11C21AB6AEB
:10263800E369013B9B000B402C3999400B00216E4C
:10264800BEE71223A26D9A43023B1343A3650123FD
:10265800E26D1343E36501230193C0E7A36D1A43B9
:10266800A265F8E7FDFEFFFF0102FEFF02FCFF1F67
:1026780008270140FFFFC3FFE8FFFF6F00000020AD
:10268800400D03007047704710B5806AFFF7FBFFE5
:1026980010BD70474023806A10B5826D134383656F
:1026A8000423C26D1343C365FFF7F3FF10BD000099
:1026B800502370B5846AA26D1A422DD1A26DB13330
:1026C800FF331343A365C02325681B01EA681A4238
:1026D80015D1A37E002B12D12B681B070FD528001C
:1026E800FFF7BCFE00280ED10C226B6893436B6089
:1026F800A26D0F4B1A400433FF331343A365200028
:10270800FFF7C0FF70BD2023A26D1343A36501230B
:10271800E26D1343E365F2E7A36DDB0603D5200002
:10272800FFF7B7FFEEE7236D5B6B9847EAE7C04614
:10273800FEFEFFFF0023F0B585B003930300009170
:1027480054331A7804000220012A4CD00122276948
:102758001A7025682800FFF781FE002800D0E9E0FC
:10276800009B04225B6880219C4697436246009B3D
:1027780009061B68022A00D1B0E05A03520B8F42A7
:1027880033D1A96A0A43AA62009A68699268190251
:102798006B4E0A403240884302436A61002B1EDABE
:1027A800E021684A6848156849042940834200D0F6
:1027B8007EE080200004054211D11368634D2B4050
:1027C8000B431843624B106018686249FDF7A6FC7A
:1027D800431C0C2058430390039B002B64D100201A
:1027E80000235434237005B0F0BD1F2167460F4005
:1027F8001039B940CE430196266E8E433100002A27
:1028080012D1980E1F321040B84062460843920811
:10281800E169013220668A42B6D8A96A01989A000D
:10282800120FBA400140ADE701221342ECD19218D1
:1028380001201342E8D1100002321342E4D10130E2
:102848001A07E1D40130DA06DED401309A06DBD467
:1028580001305A06D8D401301A06D5D40130DA0529
:10286800D2D401309A05CFD401305A05CCD40130E6
:102878001A05C9D40130DA04C6D401309A04C3D485
:1028880001305A04C0D401301A04BDD40130DA032F
:10289800BAD401309A03B7D480221800D20210406B
:1028A8001342B1D01220AFE7039B013B039393E798
:1028B800294883420BD180204004054200D08EE78E
:1028C8001368224D2B400B431843106087E72348B9
:1028D800834200D083E78020C003EEE78F4204D113
:1028E800AA6A5903490B8A43AA62002B00DB76E7E0
:1028F800144A15481168834208D1A02310685B0464
:102908000B40124901400B43136068E712488342A9
:1029180003D1C02310681B04F2E71048834200D09B
:102928005DE7C0204004136801400848034019438C
:10293800116054E72023A26D01201343A3654FE7DC
:1029480000FFFF0708270140001000B0FFFF3FFE0F
:1029580000000020400D0300004000B8002000B433
:1029680070B5056804002800FFF778FD002801D13C
:10297800002070BDAB689B0705D4AA680F4B1A40AE
:1029880010231343AB60FFF763FD0426050023689B
:102998009B683342ECD0FFF75BFD401B0228F6D959
:1029A80023689B683342F2D010230120A26D1343A1
:1029B800A365E36D0343E365DBE7C046E8FFFF7FFC
:1029C8000023F7B5026801939168013304001942A6
:1029D80001D00020FEBD90682249084208D010228C
:1029E800A16D0A43A265E26D13430120E365F1E797
:1029F80091681D4F39400B4393601C4B1B681B02A9
:102A080021D4637E012BE4D0FFF722FD01250600C7
:102A1800226813682B42DCD193682B4203D1936858
:102A28003B402B439360FFF713FD801B0228EFD92F
:102A380023681B682B42EBD11023A26D1343A365B7
:102A4800E36D2B43D1E70A4B0A491868FDF766FB8B
:102A580001300190019B002BD3D0019B013B0193D6
:102A6800F8E7C04617000080E8FFFF7F082701400D
:102A780000000020400D0300F7B505680400280099
:102A88000E000192FFF7EAFC022300283FD127003D
:102A980054373A78012A3AD0013B3B70EA681A4227
:102AA8000CD1AA681A4205D0AA681A4B1A40022308
:102AB8001343AB600123EA681343EB602000FFF780
:102AC8007FFF031E23D1A16D134A114080225200BB
:102AD8000A43A265E065114A206D2168C262104A66
:102AE8000263104A42631C220A603B704A68103332
:102AF80013434B603200019B403100F0C7F90300DB
:102B08002068044A8168114004220A438260180040
:102B1800FEBDC046E8FFFF7FFEF0FFFFB9260008B4
:102B2800912600089D2600080122036870B504005C
:102B380098689968114201D1002070BD02210842AD
:102B4800FAD105209D680540012D1ED19A681348C9
:102B580002401143032299601A60FFF779FC0600CE
:102B680023689B682B42E7D0FFF772FC801B022882
:102B7800F6D923689B682B42F2D01023A26D134329
:102B8800A365E36D2B43E36506E01023A16D0B43BA
:102B9800A365E36D1A43E2650120CEE7E8FFFF7FF6
:102BA80070B506005436337804000225012B26D070
:102BB80001233370FFF7D4FE051E1ED1206D831D3F
:102BC800DB7F022B08D100F0A9F9002804D04023AC
:102BD8000500A26D1343A3651021226820005368E5
:102BE8008B435360002D0CD1FFF79EFF051E0BD0C1
:102BF80001212268D3688B43D360002333702800F7
:102C080070BDFFF791FFF3E7A26D034B1A40043341
:102C1800FF331343A365EBE7FEFEFFFF10B5FF2468
:102C280003220B0021000240D20091409B01234067
:102C3800C943934000280ADBC0240B4A800880005F
:102C48008018A40002590A401343035110BD0F22F3
:102C580010400838054A800880008018C269114071
:102C68001943C161F2E7C04600E100E000ED00E071
:102C7800002805DB1F2318401E3B8340014A1360D0
:102C88007047C04600E100E0002809DB1F23184018
:102C98001E3B8340034AD367BFF34F8FBFF36F8F49
:102CA8007047C04604E100E08022431E5204012020
:102CB80093420DD2C021074A07485360036A0906A8
:102CC8001B021B0A0B43036200200723906013605A
:102CD8007047C04610E000E000ED00E0F0B5846CFD
:102CE800C56C6560046D002C02D0446D856D65600F
:102CF8001C24056C084E25401B3CAC4077683C43BF
:102D08007460046863608368102B02D1A260E1607C
:102D1800F0BDA160E260FBE70000024010B50400CE
:102D2800036C094A9B089B189B00436400681421A4
:102D3800C0B20838FDF7F2F9044BA3641F2318400A
:102D48001E3B8340E36410BD0082001080080240EF
:102D5800F8B504000120002C46D02568254B142125
:102D6800E818FDF7DBF902238000A61D2064F3773D
:102D78002B68214AA76813402B60E36821693B430D
:102D88000B4361692A680B43A16920000B43E16981
:102D98000B43216A0B4313432B60FFF7BFFF8023CC
:102DA800DB019F4201D1002363603F236268616CAD
:102DB80013400B60E06CA16C013A4860032A14D8F8
:102DC8000E4A0F4899180122013B9A40A265130048
:102DD80000228900216560650A60436000200123A4
:102DE800E0630534F377E077F8BD00232365636576
:102DF800A365F3E7F8FFFDBF0F80FFFF3F820010D8
:102E080040090240F8B5012504002800002C34D000
:102E1800276814213B680026AB433B60174BF81822
:102E2800FDF77CF91C238000206418402B008340A8
:102E3800134A3E60516820000B435360FFF76EFF52
:102E4800636CE26C1E60A36C5A6063685A1E032AA6
:102E580006D895400B495B189B001E600A4B5D60C5
:102E68000020A31D20656065A065E06220636063A3
:102E7800A063E0630534D877E077F8BDF8FFFDBFBD
:102E8800000002403F82001040090240F7B5451D8E
:102E98000193EE7F04000220012E33D00138E87739
:102EA800A71DFE7FB4466346F6B20096002683420D
:102EB80030D10130F8772568E6632868009B98438D
:102EC8002860019B2000FFF709FF236BB3421AD04B
:102ED8000E232A6813432B60636C1A68D20304D547
:102EE8008022196852000A431A60236D002B04D00F
:102EF8008022196852000A431A60012300202A68B8
:102F080013432B60FEBD04222B6893432B602A6871
:102F18000A23DFE78023E363EE77F3E7F0B50028C1
:102F280008D0841DE37F411D022B05D00423C36311
:102F38000023CB770120F0BD0E250268466C13688C
:102F4800AB4313603368104D2B4033600123166880
:102F58009E431660026C1B331A401B3B93400B4E7A
:102F680077683B437360C26C836C5A60036D002BB7
:102F780005D01A682A401A60436D826D5A60012391
:102F88000020E377C877D6E7FFFEFFFF0000024086
:102F9800F8B5811DCB7F022B03D00423C363012026
:102FA800F8BD0E2402681C271368456CA343136000
:102FB800012314689C4314602A68104C22402A603C
:102FC800026C0F4D3A4093406E6833436B60C26C9D
:102FD800836C5A60036D002B05D01A6822401A6072
:102FE800436D826D5A6001230022CB77431DDA7747
:102FF800836B934200D098470020D1E7FFFEFFFF84
:1030080000000240F8B51C240427016C264A214020
:103018003C008C40166803681D6826420FD03D426C
:103028000DD01968890602D41968B9431960536824
:103038001C43036B5460002B1BD0984719E00227F0
:103048003C008C40264215D03D4213D019688906B1
:1030580006D40A251968A94319600121831DD97767
:1030680053681C4354600022431DDA77C36A9342B5
:10307800E3D1F8BD082427008F403E42F9D025420D
:10308800F7D00E251C68AC431C6001231D008D4041
:103098002900546821435160821DC363D3770022FD
:1030A800431DDA77436BE2E7000002400630C07F39
:1030B800C0B27047C06B70470020054B5A69824206
:1030C80005DA044A9A60044A9A605869C00F704742
:1030D8000020024023016745AB89EFCD8022044BD5
:1030E800120659690A435A615869C043C00F7047AC
:1030F80000200240F8B505008027FFF7A9F97F02F4
:103108004619124C23693B420BD12269104B11001E
:103118001048194020611A4209D00F4B012059600C
:1031280004E0FFF795F9B042EBD30320F8BDFFF7B1
:103138008FF980264519F60223691800304033427A
:10314800F4D0FFF785F9A842F6D3EEE70020024055
:10315800FA830000FB830000EC020020F7B5174E4D
:103168000193337804000D0002200092012B1ED039
:103178000123FA203370002380007360FFF7BAFF41
:10318800002812D10E4F012C12D17B6923437B6199
:10319800009B2B60BFF36F8F019B6B60FA20800050
:1031A800FFF7A8FF7B69A3437B6100233370FEBD53
:1031B8002800009903F07CF9F0E7C046EC020020F3
:1031C80000200240044A05485369C90003401943D6
:1031D800034B0B43536170470020024007E0FFFF99
:1031E80002000100F7B5214F05003B780224019148
:1031F800012B1AD00123FA203B70002380007B604A
:10320800FFF778FF041E0ED104236B602B68042B94
:103218000DD1FA20164A174B516980000B435361B0
:10322800FFF768FF040000233B702000FEBD012368
:10323800019A5B421360AE68AB68EA689B18B342B8
:103248000CD968683100FFF7BDFFFA208000FFF74E
:1032580051FF002808D00400019B1E600221044A87
:1032680053698B435361DEE70136E5E7EC02002042
:1032780000200240040001000023F0B585B00A6870
:103288001400DC4001D105B0F0BD012514009D40BB
:103298002C4000942A4200D191E04A685F0094468D
:1032A8000322644622400324BC40E4430194541E94
:1032B800012C2ED88668019C2640CC68BC4034433B
:1032C800846044680126AC432500644624093440E0
:1032D8009C402C434460C568019C25408C68BC40D8
:1032E8002C43C460022A16D107250F261D40AD00C5
:1032F800AE40DC08A40004190294246A0396260050
:10330800039CA64334000E69AE402643029C266205
:1033180001E0032ADFD1BA400468019D25402A4311
:10332800C02402606246A402224248D0254A0325EE
:103338009C08A400A4180F221D40ED00AA40A02755
:10334800266EFF0596430022B8420CD01E4F01326C
:10335800B84208D01D4F0132B84204D01C4F033286
:10336800B84200D1023AAA40674632432266154C59
:10337800009A2668009DD2433543FF0201D43500E8
:103388001540674625606668009D3543BF0201D435
:1033980035001540674665600E4C009DE66F354365
:1033A800BF0301D4350015406746E5670A4C009E07
:1033B800E56F2E43FF0301D415402E00E667013365
:1033C8005DE7C046001802400004005000080050A5
:1033D800000C00500818024004180240F0B5002301
:1033E8000F0085B03A00DA4001D105B0F0BD0122E6
:1033F8009A40140001923C40174253D02A490325B1
:103408009A08920052180F211D40ED00A940166E2F
:1034180002910E400396A0260021F605B0420FD077
:1034280022498C46012160450AD021498C46022157
:10343800604505D01F498C460321604500D0023104
:10344800A940039DA94212D11B4E1749F56FA54308
:10345800F5671A4EF56FA543F5674D68A5434D60AE
:103468000D68A5430D60116E029CA14311660324EB
:1034780059008C4007210F26194089008E400268A8
:10348800019922430260DA0892008218156AB5434E
:1034980015628268A243826042688A434260C268B9
:1034A800A243C26001339DE70018024000040050A7
:1034B80000080050000C0050041802400818024090
:1034C80000690840431E9841C0B27047002A01D0E5
:1034D800816170478162FCE7426913000B401B045D
:1034E80091430B438361704770B5084D0400EB6846
:1034F800184202D0E86002F047F92B69234203D052
:1035080020002C6102F0FEF970BDC0460018024090
:1035180070B504000120002C16D02368124A072633
:103528001A60124A1A6062685A60A2689A60FEF7C6
:103538008FFF05002368DA68324206D11969E2680C
:1035480091420DD01A61002070BDFEF781FF401B2B
:103558003128EFD92368DB683342EBD00320F3E747
:10356800034A1A60EFE7C046CCCC0000555500006E
:10357800AAAA00000368024A00201A607047C046E1
:10358800AAAA000010B5114C1149236802000B408B
:1035980003432360802300209B009A420ED10D4BE9
:1035A8000D49186806235843FCF7B8FD8022431CD0
:1035B800D200616908001040114200D110BD002BF3
:1035C80001D0013BF5E70320F8E7C0460070004052
:1035D800FFF9FFFF0000002040420F00F0B5040093
:1035E80085B0002802D1012005B0F0BD0368DB07D3
:1035F80010D423689B075CD423681B0700D5C1E05F
:1036080023685B0700D5F2E0E369002B00D079E17D
:103618000020E9E73822AF4DAB681340EA68102B69
:1036280009D1D3439B0708D12B689B03E1D5636875
:10363800002BDED1D7E7082BF6D080226368520230
:10364800934211D12A6813432B60FEF701FF8027AC
:103658000600BF022B683B42CBD1FEF7F9FE801B68
:103668006428F7D90320BFE7A021C9028B4208D1FB
:1036780080232968DB020B432B602B681A432A60DE
:10368800E3E72A6894490A402A602A6893490A406D
:103698002A60002BD9D1FEF7DBFE80270600BF0287
:1036A8002B683B42A5D0FEF7D3FE801B6428F7D9D0
:1036B800D8E73822874DAB681340EA68102B28D129
:1036C80003210A40022A26D12A68520503D5E26856
:1036D800002A00D187E769686269814812020140BF
:1036E8000A436A60002B0CD12B687E4A7E4913403E
:1036F800226913432B602B687C4A9B045B0FDA40DA
:103708000A607B4B1868FEF75BFE002800D173E760
:1037180069E7002BD8D0E368002B20D02B68714ACA
:10372800802713402269FF0013432B6080232A68F7
:103738005B0013432B60FEF78BFE06002B683B42B1
:1037480007D06A68636966491B020A4013436B60C5
:1037580052E7FEF77DFE801B0228EFD982E72B682F
:10376800644A802713402B60FEF772FE0600FF00B4
:103778002B683B4200D13FE7FEF76AFE801B022818
:10378800F6D96FE73822534DAB681340182B08D190
:103798002B6E9B0700D433E7A369002B00D02FE7DB
:1037A80021E7A2690123002A10D02A6E02271343B9
:1037B8002B66FEF74DFE06002B6E3B4200D01FE73E
:1037C800FEF746FE801B0228F6D94BE72A6E022731
:1037D8009A432A66FEF73CFE06002B6E3B4200D158
:1037E8000EE7FEF735FE801B0228F6D93AE73822A5
:1037F800384DAB681340202B08D1EB6D9B0700D4E4
:1038080002E7A368002B00D0FEE6ECE68022002148
:10381800EB6B52050091134208D1EB6B1343EB633A
:10382800EB6B13400393039B012300938027324ED5
:103838007F0033683B4215D0A368012B22D1EA6D83
:103848001343EB65FEF704FE02270600EB6D3B42CF
:1038580038D0009B012B00D0D6E6EB6B274A1340EB
:10386800EB63D1E633683B433360FEF7F1FD01902B
:1038780033683B42E0D1FEF7EBFD019BC01A0228FA
:10388800F6D9EFE6EA6D052B05D1013B1343EB654D
:10389800EA6D0123D4E701218A43EA65EA6D033121
:1038A8008A43EA65002BCDD1FEF7D2FD0227060038
:1038B800EB6D3B42CDD0FEF7CBFD114B801B984200
:1038C800F6D9CFE6FEF7C4FD0D4B801B9842BDD953
:1038D800C8E6C04600100240FFFFFEFFFFFFFBFFE7
:1038E800FF80FFFFFFC7FFFF000000200024F40057
:1038F80008000020FFFEFFFF00700040FFFFFFEF01
:103908008813000038213F4DAA680A40102A51D078
:103918003D4A022B38D12B68802713402B60FEF7D5
:1039280097FD0600BF042B683B4227D1616A236AD2
:10393800EA680B43354980260A401343E26AB60415
:103948001343226B1343A26A12021343EB608023D2
:103958002A685B0413432B608023EA685B051343E2
:10396800EB60FEF775FD04002B68334200D04FE68C
:10397800FEF76EFD001B0228F6D973E6FEF768FD18
:10398800801B0228CFD96DE62B68802613402B6058
:10399800FEF75EFD0400B6042B68334204D1EB68E1
:1039A8001B4A1340EB6033E6FEF752FD001B02286A
:1039B800F2D957E6012B00D115E60322E868216AFF
:1039C80002408A4200D00EE67022616A02408A42B2
:1039D80000D008E6FE21A26AC90101401202914204
:1039E80000D000E6F822E16A920302408A4200D041
:1039F800F9E5236B400F4007C01A431E9841C0B237
:103A0800F2E5C04600100240FFFFFFFE8C80C11F98
:103A1800FCFFFEEF382370B51D4CA2681A4205D191
:103A280023681C489B045B0FD84070BDA2681A40ED
:103A3800082A27D0A2681A40102A17D1E368E1683B
:103A4800DB43E5684906490F6F322D0A01311540FD
:103A58009B0709D11048FCF761FBE1686843490FEF
:103A68000131FCF75BFBE0E70A48F4E7A2681A407B
:103A7800202A09D0A26800201340182BD5D1FA209B
:103A8800C001D2E70448D0E780200002CDE7C04655
:103A9800001002400024F40000127A00F7B5040078
:103AA8000D00002801D10120FEBD07274A4E3368CA
:103AB8003B408B422AD3226893073BD4D20748D491
:103AC800072733683B40AB420AD93368BB432B43D3
:103AD8003360FEF7BDFC019033683B40AB426BD1CD
:103AE80023683E4D5B076FD4FFF794FFAB683C49F2
:103AF8001B051B0F9B005B581F210B40D840394A00
:103B0800394B10601868FEF75BFCCDE73368BB43A0
:103B18000B433360FEF79CFC019033683B40AB429B
:103B2800C9D0FEF795FC019BC01A304B9842F4D9D6
:103B38000320B9E72949530704D5E0238868DB0146
:103B480003438B608B682A480340A06803438B605B
:103B5800B4E76268214F012A19D13B689B03A2D5BB
:103B68000721BB688B431343BB60FEF771FC0190D0
:103B78003823BA681A406368DB009A42A0D0FEF77F
:103B880067FC019BC01A194B9842F1D9D0E7022A69
:103B980003D13B689B01E3D485E7002A03D13B6846
:103BA8005B05DDD47FE70223032A03D1396E19426E
:103BB800D6D178E7F96DFAE7FEF74AFC019BC01AFF
:103BC8000A4B984288D9B3E7AB680A4A1340E268BF
:103BD8001343AB6088E7C046002002400010024053
:103BE800E864000800000020080000208813000096
:103BF800FFF0FFFFFF8FFFFF064B07499B68074A4F
:103C08005B045B0F9B005B581F2110680B40D8407A
:103C18007047C04600100240C86400080000002039
:103C2800F0B50368050085B000209B0351D58022BC
:103C3800484C5205E36B0090134208D1E36B1343E1
:103C4800E363E36B13400393039B012300938027F3
:103C5800414E7F0033683B433360FEF7F9FB019028
:103C680033683B4227D0E16DC022080092006B699F
:103C78001040114217D098420CD0E36D374AE16DDD
:103C88001340802252020A43E265E26D34490A4039
:103C9800E265E365DB0706D5FEF7DAFB02270600D7
:103CA800E36D3B424ED0E36D2C4A002013406A6915
:103CB8001343E36506E0FEF7CBFB019BC01A02281D
:103CC800CED90320009B012B03D1E36B254A134077
:103CD800E3632A68D30706D503241E494B6DA34323
:103CE8006C6823434B65930606D51A491E4C4B6DE9
:103CF8002340AC6823434B6553040FD515492C6901
:103D08004B6D9B009B0823434B658023DB059C423E
:103D180004D18023CC685B022343CB6012050FD506
:103D28000C4A124C536DE96823400B4353658023BA
:103D3800DB01994204D18023D1685B020B43D36035
:103D480005B0F0BDFEF784FB094B801B9842A7D94C
:103D5800B7E7C0460010024000700040FFFCFFFFBC
:103D6800FFFFFEFFFFFFFFEFFFCFFFFFFF3FFFFF5C
:103D7800881300000122036A70B593430362036A43
:103D8800164A4468856915400A6815430222934318
:103D98008A681343124A904205D0124EB04202D0AC
:103DA800114EB04213D10826B343CE6833430426DC
:103DB800B343904205D00B4A904202D00A4A90423F
:103DC80005D10A4A8E6922404C69344314434A6833
:103DD800446085614263036270BDC0468CFFFEFF8C
:103DE800002C01400044014000480140FFFCFFFF57
:103DF800036A174A70B513400362056A154B426897
:103E0800C4691C400B681C43134B1D408B681B0284
:103E18002B43124DA8420ED1114D1D40CB681B02F9
:103E28002B43104D2B40104D4E6915408A69324383
:103E380012012A4305E00D4DA842F4D00C4DA842CA
:103E4800F1D042604A68C461C263036270BDC04673
:103E5800FFFEFFFF8CFFFEFFFFFDFFFF002C014070
:103E6800FFF7FFFFFFFBFFFFFFCFFFFF004401400D
:103E780000480140036A124A30B513400362046ADD
:103E8800104D4368C2692A400D682D0215430E4A39
:103E980014408A68120322430C4CA04205D00C4CF3
:103EA800A04202D00B4CA04204D10B4C1C404B69E1
:103EB8009B01234343604B68C5610364026230BDC4
:103EC800FFEFFFFFFF8CFFFEFFDFFFFF002C01402D
:103ED8000044014000480140FFBFFFFF036A70B57E
:103EE800104C114A23400362066A4368456D154029
:103EF8000A6815430D4A16408A68120432430C4E6C
:103F0800B04205D00B4EB04202D00B4EB04203D1A6
:103F18001C404B691B02234343604B68456583651E
:103F2800026270BDFFFFFEFF8FFFFEFFFFFFFDFF78
:103F3800002C01400044014000480140036A124A35
:103F480030B513400362046A104D4368426D2A403D
:103F58000D682D0215430E4A14408A681205224343
:103F68000C4CA04205D00C4CA04202D00B4CA042F5
:103F780004D10B4C1C404B699B02234343604B68A4
:103F88004565C365026230BDFFFFEFFFFF8FFFFE8F
:103F9800FFFFDFFF002C01400044014000480140C2
:103FA800FFFFFBFF01000300012010B53D310C7835
:103FB800E2B2844218D1001808701B68D96811430E
:103FC800D9600B498B4202D00A498B420DD19A68BD
:103FD80009490A40062A06D007398A4203D0012235
:103FE80019680A431A60002010BD1968F9E7C0462D
:103FF800002C014000040040070001007047000049
:10400800194A10B50368904202D0184CA04208D152
:104018007024A3434C68234390420BD0134CA04216
:1040280008D0134CA04205D0124CA04202D0124C2A
:10403800A04203D1114C1C40CB6823438024A343E6
:104048004C69234303608B68C3620B6883629042A8
:1040580005D0084B984202D0074B984201D10B6912
:1040680003630123436110BD002C0140000400409C
:10407800002000400044014000480140FFFCFFFFD1
:1040880070B504000120002C23D025003D352B7885
:10409800DAB2002B05D123003C3320001A70FEF75A
:1040A80013F802232B702068211DFFF7A9FF2200B7
:1040B800012300204832137047340A3A13705370B2
:1040C8009370D370137153719371D37113722370FA
:1040D8002B7070BD70B504000120002C23D0250082
:1040E8003D352B78DAB2002B05D123003C33200074
:1040F8001A70FFF783FF02232B702068211DFFF73A
:104108007FFF2200012300204832137047340A3A07
:10411800137053709370D370137153719371D3717B
:10412800137223702B7070BD1022036A70B593430D
:104138000362056A154C4268836923400C682402AF
:104148001C4320239D438B681B012B43104DA84221
:104158000FD18025AB431E00CB68403D1B01334384
:10416800AB430C4D4E6915408A69324392002A438D
:1041780005E0094DA842F4D0084DA842F1D04260AC
:104188004A6884618263036270BDC046FF8CFFFE8B
:10419800002C0140FFF3FFFF0044014000480140AC
:1041A800F8B507003C3715003A7803000C000220E8
:1041B800012A0CD0013838700C2D51D008D8042DA4
:1041C8002DD0082D3CD0002D17D000233B70F8BD12
:1041D800102D58D0142DF8D11D682800FFF7AEFE19
:1041E80080236A6D1B0113436B656B6D2E4A134068
:1041F8006B6523696A6D1B0253E01D682800FFF791
:10420800B9FD0823AA6913430422AB61AB69934340
:10421800AB61AB6922691343AB610020D5E71D6828
:104228002800FFF781FF8023AA691B011343AB61B4
:10423800AB691D4A1340AB612369AA691B02EAE70F
:104248001E683000FFF7D4FD0422F3691D43F561B1
:10425800F3699343F361F36922691343F361DCE77C
:104268001D682800FFF706FE8023EA691B01134337
:10427800EB61EB690C4A1340EB612369EA691B02A5
:104288001343EB61C9E71D682800FFF727FE0823E1
:104298006A6D134304226B656B6D93436B656B6D9D
:1042A800226913436B65B8E7FFFBFFFF1F2310B5B7
:1042B800012419408C408A40036AA3430362036ABD
:1042C8001A43026210BD000010B508291CD006D898
:1042D80000290BD0042914D00300433308E00C292B
:1042E80015D01029F8D10300423301E003003E3312
:1042F8001B78013B5A1E9341DBB2002B0AD00120E8
:1043080042E003003F33F3E703004033F0E70300E4
:104318004133EDE7022308293ED009D800290ED001
:10432800042932D00200433213700429E7D12FE068
:104338000C2939D01029F5D142300370DFE702008B
:104348003E3213700468E2681343E3600468012294
:104358002000FFF7ABFF1C4A94422DD01B4B9C4218
:104368002AD01B4B9C4227D01A4B9C4207D1A368EA
:10437800194A1340062B06D0073A934203D001236B
:10438800226813432360002010BD02003F321370DF
:1043980002680423D4680DE00200403213700268FA
:1043A800D3680B43D360D1E7020041321370102366
:1043B8000268D4682343F5E78023616C1B020B4332
:1043C80063649442D3D0CFE7002C014000440140FD
:1043D80000480140000400400700010010B5FFF745
:1043E80073FF10BD30B5EFF31084012282F31088FB
:1043F800C02501680B68AB430B6084F31088EFF3AA
:10440800108182F310880268044C936823409360FB
:1044180081F3108820238830036030BDFFFF7FFFC1
:1044280030B5EFF31084012282F310880168134D30
:104438000B682B400B6084F31088EFF3108182F334
:10444800108802680E4C93682340936081F31088AB
:10445800C36E012B0AD1EFF3108183F31088102467
:1044680002681368A343136081F3108803002022B5
:104478008C331A600023C366436730BDDFFEFFFF3D
:10448800FEFFFFEF70B505000120002D19D02E00AA
:1044980024230024883633602B681A6882431A6004
:1044A80028001C605C609C60FDF73EFF2B0020002C
:1044B80090331C60043B34601C60EC662C678435C8
:1044C8002C7070BDF7B50500883513002A68040004
:1044D8000220202A04D1002901D0002B01D101207B
:1044E800FEBD8022A0685201904204D12269002AB0
:1044F80001D1CA07F3D422002600543221650027CF
:1045080013805380212290363760E06F2A6022683A
:104518000192B84211D0114A8763C262104A0263FD
:10452800104A4263019A2832FEF7B0FCB84204D020
:1045380010233360DB182B60D1E7402223681A620E
:10454800EFF31081012383F3108822687F3390688A
:104558000343936081F310880020C1E719460008DF
:104568006B4600087B4600080300020080218C325D
:10457800883370B51B6815680268040092680A429F
:1045880020D0212B1ED1EFF31080203B83F310881D
:10459800226893688B43936080F31088E06F00284B
:1045A8000DD0FEF7BBFC002809D0E06FFEF782FDB6
:1045B800202804D110239034032023600AE020002F
:1045C800FFF710FF402123689B680B4201D0222D82
:1045D80001D0002070BDEFF31080012383F3108811
:1045E800250004CD93688B43936080F31088E86FAF
:1045F800002808D0FEF792FC002804D0E86FFEF7E8
:1046080059FD2028D6D02000FFF70AFFE1E77047C0
:1046180003001B6870B51A6820231100806A1940CE
:104628001A421AD1030056331980EFF3108401227D
:1046380082F31088802501688B68AB438B6084F314
:104648001088EFF3108182F3108840230268106805
:104658000343136081F3108870BDFFF7D8FFFBE7B1
:10466800704710B5806AFFF7FBFF10BD70477047B1
:10467800704770B5846A230088331A685D682368B8
:104688009B681B0608D5212A06D123000022563331
:1046980020001A80FFF7A6FE23689B685B0608D5F2
:1046A800222D06D1230000225E3320001A80FFF756
:1046B800B7FE220010239032116820000B431360CC
:1046C800FFF7D6FF70BD806A0023020010B55E3286
:1046D8001380083A1380FFF7CBFF10BD7047000026
:1046E800F7B50168C14DCB6904000A6888682B4298
:1046F80010D120252B4200D19BE08026760515405D
:104708000640354300D194E0636F2000002B00D0B1
:1047180085E085E0B64D05400095B64D009E1540F4
:10472800354300D185E0250001269035334205D078
:10473800D70503D50E622F683E432E60022633420A
:104748000CD0C7070AD527000E6290373E6801973C
:10475800B446042667463E43019F3E600426334222
:104768000CD0C7070AD527000E6290373E6801971C
:10477800B446022667463E43019F3E600826B4467B
:10478800334209D02027009E1740374304D066469D
:104798000E622F683E432E6080263601334206D0D3
:1047A800570104D50E6220212E68314329602968FB
:1047B800002935D020210B420AD080235B05114007
:1047C8000340194304D0636F002B01D020009847A1
:1047D80022682B684027966828223E401340200014
:1047E8001E4322D0FFF71CFE23689B683B4218D06B
:1047F800EFF31081012383F31088250004CD93681B
:10480800BB43936081F31088E86F002809D07A4B86
:104818008363FEF7BDFB002802D0E86F836B9847DF
:10482800F7BD2000FFF724FFFAE7FFF721FF2E600E
:10483800F6E7E56E012D00D09FE01026334200D147
:104848009BE0324200D198E00E62896840230A005A
:104858001A40194257D0211DCA6F1068426892B297
:10486800002ADDD027005C373F889742D8D9270037
:104878005E373A80026820208446104000906046E7
:10488800024232D1EFF3108785F3108820685B4E1F
:1048980002683240026087F31088EFF3108785F3CF
:1048A800108820688268AA43826087F31088EFF333
:1048B800108785F31088206882689A43826087F39E
:1048C8001088230062468C331A60009BE366EFF37E
:1048D800108085F3108822680F351368AB43136086
:1048E80080F31088C86FFEF719FB022322002367A4
:1048F80023005C325E331B881188C91A89B22000F4
:10490800FFF7ECFE8CE7230020005C335E3019884B
:10491800038800889BB2002800D181E7C91A89B2B0
:10492800002900D17CE7EFF3108785F31088206811
:10493800334E03683340036087F31088EFF3108722
:1049480085F3108820682F4E83683340836087F38F
:104958001088230020208C331860E2666267EFF32A
:10496800108085F31088102522681368AB43136004
:1049780080F3108802232367C1E780256D032B424B
:1049880006D0460204D520000D6200F03FFB47E741
:1049980080210B4207D080252D0411402840014377
:1049A80001D0A36FB1E640210B4216D00A4214D0C1
:1049B800EFF31080012383F31088226813688B4378
:1049C800136080F310882300202288331A600023A4
:1049D8002000A367FFF71BFE22E7190214D5510038
:1049E80012D5200000F014FB1AE7C0460F0800009B
:1049F8000100001020010004CF460008FFFEFFFF61
:104A0800DFFEFFFFFEFFFFEFDB0100D408E7002A0F
:104A180000DB05E7200000F0FAFA01E70123806ACD
:104A280010B50367C36E012B06D103005C331988E8
:104A38004908FFF753FE10BDFFF719FEFBE700001A
:104A480003001B6820221B6870B51900806A11409A
:104A5800134234D103005E331980EFF3108501232C
:104A680083F3108804681D4E21683140216085F366
:104A78001088EFF3108583F310880468A1689943C0
:104A8800A16085F31088EFF3108483F31088402524
:104A980001688B68AB438B6084F3108803008C3308
:104AA8001A60C36E012B0AD1EFF3108183F31088CB
:104AB800102402681368A343136081F3108800234D
:104AC8000367C36E012B05D103005C331988FFF718
:104AD80005FE70BDFFF7CAFDFBE7C046FFFEFFFFFE
:104AE80070B504002569A168036829436569C2692E
:104AF80029431868494D11432840014319605968F2
:104B08004748256A0140E06801435960A1699868EF
:104B18002943444D284001430F209960D96A8143B5
:104B2800606A0143D96240498B4215D103213F4B4A
:104B38005B6D0B40013B022B60D83D49C85C80236C
:104B48001B029A422FD1082856D8FBF7DDFA5B558D
:104B58000E550B5555550F0036495B18591E8B419C
:104B68001801ECE7FEF756FF4EE0334A616A334B13
:104B780049001000C95AFBF7D1FA656840006B0874
:104B8800C0182900FBF7CAFA02002D4B103A9A42C6
:104B980032D80F23020000079A4393B2400F2268CD
:104BA8000343D36032E0082826D8FBF7ADFA1A256C
:104BB80005251F25252522001F48626A1F4B520024
:104BC800D15AFBF7ABFA65686B08C0182900FBF7E8
:104BD800A5FA02001A4B103A9A420DD82368D860F9
:104BE80014E0FFF709F8002810D0E6E7FEF712FFF7
:104BF800F9E780200002E0E7012008E080231B029B
:104C08009A42EED1FEF7F8FF021EAFD100200D4BFD
:104C1800A36600236367A36770BDC046F369FFCF2F
:104C2800FFCFFFFFFFF4FF110038014000100240E2
:104C38002865000800BCFFBF0024F4002C650008AC
:104C4800EFFF000001000100836A30B5DA0706D5DE
:104C58000168284C4A682240C46A22434A609A077D
:104C680006D50168244C4A682240046B22434A60F6
:104C78005A0706D50168214C4A682240446B2243F2
:104C88004A601A0706D501681D4C4A682240846BA1
:104C980022434A60DA0606D501681A4C8A6822401F
:104CA800C46B22438A609A0606D50168164C8A6846
:104CB8002240046C22438A605A0610D50168134DBD
:104CC8004A68446C2A4022434A6080225203944234
:104CD80005D14A680E4C2240846C22434A601B0668
:104CE80006D502680B4953680B40C16C0B435360EF
:104CF80030BDC046FFFFFDFFFFFFFEFFFFFFFBFFCC
:104D0800FF7FFFFFFFEFFFFFFFDFFFFFFFFFEFFF6B
:104D1800FFFF9FFFFFFFF7FFF8B504000D00170026
:104D28001E002268D3692B405B1B59424B41BB4292
:104D380001D0002029E0069B0133F3D0FDF788FB62
:104D4800069B801B984201D8002B1FD1EFF31080DF
:104D5800012282F310882168204D0B682B400B60DC
:104D680080F31088EFF3108082F3108821688B6835
:104D780093438B6080F3108823001F3288331A60B6
:104D88005A600023032084342370F8BD23681A680E
:104D98005207C6D58022D96912011142C1D01A62C0
:104DA800EFF31080012282F3108821680B4D0B6805
:104DB8002B400B6080F31088EFF3108082F310888B
:104DC80021688B6893438B6080F31088220020232E
:104DD8008832136053609360D3E7C0465FFEFFFFDD
:104DE800030073B50026040090331E60FDF730FB06
:104DF800236805001B681B0719D423681B685B0719
:104E08000AD58021104B0022009320002B00C903F3
:104E1800FFF782FF002815D12200002020238832C6
:104E280013605360E0662067843420700BE08021B3
:104E3800054B32000093890303002000FFF76CFF45
:104E48000028DAD0032076BDFFFFFF0170B5041EED
:104E580001D1012070BD050088352B68002B04D1D5
:104E6800020084321370FDF7DDF924230121226842
:104E78002B60136820008B431360FFF731FE012875
:104E8800E7D0A36A002B02D02000FFF7DDFE2368DD
:104E980007495A6820000A402A215A609A688A43BA
:104EA8009A60012219680A431A60FFF799FFD1E74F
:104EB800FFB7FFFFF8B513000200060005005C32DB
:104EC80081650F0013802221002290368C353260D4
:104ED8002960011D0400C86F904213D01D498263E8
:104EE800C1621D493A0001631C49416321682431AC
:104EF800FDF7CCFF002805D0102301203360DB1814
:104F08002B60F8BD2369002B0BD0EFF31081012330
:104F180083F310882268FF3310680343136081F31A
:104F28001088EFF31080012383F3108821688A68C2
:104F38001A438A6080F31088EFF3108183F3108896
:104F480022683F3390680343936081F31088002000
:104F5800D7E7C046494A0008254A00087B460008AA
:104F680003008C3070B504680220202C25D101384C
:104F7800002922D0002A20D080209C684001844249
:104F880005D11869002802D10130014215D100204D
:104F9800D8661868406800020CD5EFF31085012028
:104FA80080F3108880201C68C00426683043206085
:104FB80085F310881800FFF77DFF70BDF7B507006F
:104FC800436E04006A37002B04D10120388068340E
:104FD8002080F7BD03680B4E9A689B680A4D5B0FEB
:104FE800F05CE95CC0000192FBF722F9019B388074
:104FF8001B015B0FF05CE95CC000FBF719F980B29C
:10500800E5E7C0464C6500084465000870477047EE
:105018007047000070B50400843422780300022031
:10502800012A11D01D002422012688352A601A6819
:1050380011681068B04310600448014000205866A9
:10504800202311602B60207070BDC046FFFFFFDF7A
:10505800F8B5050084350B0029780222012915D0FE
:1050680006000121046888362232326027682268E7
:105078008A432260A168C900C9081943A160FFF7E3
:105088009DFF20230022276033602A701000F8BD9E
:10509800F8B5050084350A0029780223012915D0BE
:1050A80006000121046888362233336027682368A4
:1050B8008B432360A168064B19401143A160FFF799
:1050C8007DFF20232760336000232B701800F8BD74
:1050D800FFFFFFF100230270FA22437152000B1CFC
:1050E800914200D2131CC3807047F7B51F004900D6
:1050F80008AB1E78CBB2141E0190009316D000F0B6
:10510800C5FD009800F084FE00F004FE451E200056
:1051180000F07EFE00F0FEFD6B425D410138434227
:105128005841EDB22D182C0000F0D2FD00F0AEFD74
:1051380000980130C0B200F06BFE00F0EBFD0128D2
:1051480001D10134E4B2013EF6B2122E01D8002C8E
:1051580005D000F0BDFD019B20001C71FEBD300094
:1051680000F088FE38700137EDE7F7B50C001E0037
:1051780008AB1D780192070000F088FD6000C0B2FE
:1051880000F046FE00F0C6FD0400019800F040FE65
:1051980000F0C0FD01280ED1013C63425C4101349E
:1051A80000F096FDE0B23871FEBD307800F030FEB8
:1051B80000F0B0FD0136012CF2D0013DEDB2122D08
:1051C800F3D90024ECE7F0B5030041180825FF20C7
:1051D80031268B4200D1F0BD1A7850402A0047B2E0
:1051E8004400E0B2002F01DA7440E0B2013AD2B2D2
:1051F800002AF4D10133ECE737B5438804000A33B9
:105208009BB243800A2B5ED94279002A0CD1012334
:10521800437132330381030002320178083300926C
:10522800AA32FFF7A2FF37BD962B4CD9012A4AD1E3
:105238000223050043711C350533017800220093D1
:105248002B00FFF752FF2379002B38D106212800C5
:10525800FFF7B9FFE31CDB7F8342E4D16722237F9A
:105268009343182BDFD1A07F637F0002184340BA15
:10527800E57F80B2000228180009FBF71DFC1549DC
:10528800FBF718F9D6218905FBF714F90F232063DA
:105298001D40631CDB7FA21C2D02D07F5B191B0203
:1052A800C018FBF709FC0C49FBF704F9D62189055E
:1052B800FBF700F90949FBF73BFA6063B3E7002302
:1052C80023636363AFE7E2889A42ACD20023637139
:1052D8006380A8E70000C842000048430000484235
:1052E8001022084B10B51B6819680A431A6050222F
:1052F8001A6200F0ABFFFA2138220348C900FFF711
:10530800E9FE10BD5402002008030020F7B5294C1F
:105318000121228813004800205A984240D8051CD1
:10532800904200D9151CAAB20131FA29F3D193424F
:1053380004DD214908881B189B1A0B801F4D2B7808
:105348005A1C2A70032B2AD91D4B1B4F1C881D4B36
:1053580005211E881C4B24B21B7836B25BB2019320
:105368000023F85EFAF764FF03B218481849584357
:10537800FAF75EFF0A216043FAF75AFF019B80198A
:105388005843144B144A00B218801178012909D1E6
:105398001B88124A1BB2138000233B802B70F7BD79
:1053A8000300C1E71278002AF6D11B880C4A1BB209
:1053B800F1E7C0467C0300204A030020490300208F
:1053C800720300207003002028000020E40C000075
:1053D800FF0F00007A0300207205002078030020E8
:1053E80076030020F0B50825012602000B4F0C4873
:1053F80001390B4B89B2994200D1F0BD137858405E
:105408002B0004004008344001D0784080B2013BB2
:10541800DBB2002BF5D10132EAE7C04601A0FFFF5D
:10542800FFFF0000002130B58BB00C2207A80691C1
:1054380000F0FAFF02230293DB1803930B33049363
:105448000125274B06AC1A881B8822701B0A63703B
:10545800244B05951A881B88A2701B0AE370224BFF
:105468001A881B8822711BB21B1263711F4B1A8882
:105478001B88A2711BB21B12E3711D4B1A881B8873
:1054880022721BB21B1263721A4B1A88A2721B88F3
:105498001BB21B12E372184B1B88A381FDF70CFE8D
:1054A80001A902A8FDF79EFE002802D0FDF716FE0E
:1054B8000AE02800069A079B1049FDF74FFE0028CE
:1054C80005D0FDF70BFE032528000BB030BD2800E2
:1054D800089A099B0A49FDF741FE051EE6D0F0E748
:1054E8007005002074030020720300207003002060
:1054F8006A030020240000206603002000780008CA
:105508000878000810B5012383F31088FFF78AFF95
:10551800002383F3108810BD022330B5012487B01F
:10552800154D0293DB1803930A3304932B680594F3
:1055380008332B60FDF7C0FD104B2A689A420AD940
:105548000F4B01A902A82B60FDF74CFE002802D0E2
:10555800FDF7C4FD0CE00B4B01201A8829680023D5
:1055680092B2FDF7FBFD041EF2D0FDF7B7FD032450
:10557800200007B030BDC04620000020D8770008C2
:10558800007000086E03002010B50400A02001225E
:105598002021C005FDF79AFF220009490948FEF7B6
:1055A80091FF0948FDF782FD0128FAD1043000F087
:1055B80001FFA02000222021C005FDF787FF10BDB4
:1055C800F3050020540200209C010020F0B55D4C3A
:1055D80085B0E378A2781B021343677903935EBA18
:1055E8002379062120003F021F43FFF7FBFE030A31
:1055F800DBB20193C3B20293534B7DBA1A88534B63
:10560800B6B25A80524AADB2127852B29A80514A12
:105618001278DA80504A12881A81504A12885A81C0
:105628004F4A12889A814F4A1288DA814E4A128864
:105638001A824E4A11784E4A090212780A435A824F
:105648004C4A12889A824C4A1288DA8272190C2AB9
:1056580055DCA27902998A4272D1E27901998A428B
:105668006ED1464F227876003A706278F618002498
:105678003B007A706A00BA70E8B20233844235D1CE
:105688006400E4B2E11C3800C9B2FFF7ABFE6B005E
:10569800FB18D870AB1C000A5B000534F854E0B264
:1056A800FFF772FFFE23039A1B029A4248D1254B4B
:1056B80002999A798A4243D1DA7901998A423FD18B
:1056C8002E4C1A78052122705B782D4A6370138856
:1056D80020001B0AE37013886D00A5702371FFF783
:1056E80081FE6071000AA071072027E00021725E28
:1056F8000134111259709A70E4B20236BDE7FF23E3
:10570800039A1B029A42CDD180235B009F4217D196
:10571800A379029A934213D1E379019A93420FD164
:105728000024184D154E03E02B5D33550134E4B2C7
:105738002800FAF7E1FC8442F6D3C0B2FFF724FF51
:1057480005B0F0BD730500207A0300204C0300204B
:105758002700002026000020740300207203002088
:10576800700300206E0300206A03002068030020F5
:10577800690300202400002066030020F3050020B0
:105788006C0300200C000020F7B50400A020402185
:10579800C005FDF795FE4B4B80211870A020C00571
:1057A8000193FDF78DFE802C38D1012831D1FCF70B
:1057B8004FFE454E05003368C31A072B0FD8FA2150
:1057C8000420890000F0B8FD404F3B78012B06D13A
:1057D800FA210220490000F0AFFD00233B70019B35
:1057E80035601B78012B03D1394A137801331370C4
:1057F800384A13780133DBB21370092B09D9344BBB
:1058080035491878022807D901200870002111703D
:105818001970324BDC60F7BDFF20F6E7082CF8D191
:1058280003202F4900F088FDA0202100C005FDF7C6
:1058380047FE0128EDD12B4B2B4E2C4D2C491870CF
:105848002B880A88378812B21BB23FB29B1A294E9E
:10585800294ABB4226DD0020337810700133DBB2C1
:105868003370022B05D9254A1070FA2B01D903236E
:105878003370234B00229A5E092ACADD2B881BB29B
:10588800D8171B1843409BB29342C2DA0B881BB24D
:10589800D9175B184B409BB29A42BADD0022174BCE
:1058A8001A70B6E70027137837700133DBB213702C
:1058B800022BDED9114E3070FA2BDAD9032313707C
:1058C800D7E7C046480300204403002026000020F4
:1058D8004303002042030020280000200018024053
:1058E800881300007205002024000020780300209F
:1058F80076030020410300204003002027000020F9
:1059080066030020010010B5082807D1A020C005B3
:10591800FDF7D6FD002801D1014B187010BDC04617
:105928007205002070B5214C05002000FEF7AAFD85
:10593800012D37D0023D6B425D411D4B6842184036
:1059480096239B01C0181B4B0C2223600023606028
:105958002000A360E36023616261A361E3612362C5
:105968006362A362FFF772FA002801D0FCF736FBE6
:1059780000212000FFF76CFB002801D0FCF72EFB6C
:1059880000212000FFF784FB002801D0FCF726FB4C
:105998002000FFF73FFB002801D0FCF71FFBFFF7B3
:1059A8009FFC70BD9620C001CDE7C0465402002080
:1059B80080BB000000380140F7B5904C062165799E
:1059C80023792D021D436DBAE778ABB20193A37812
:1059D80020003F021F43FFF705FD0600884B062203
:1059E80018002100019300F04BFD019AF3B2360A2A
:1059F800F6B29371D671F0221201974229D1A27999
:105A08009A4214D1E379B34211D1ABB2013BF62BE0
:105A180011D87C4F3E883D80B6B2FFF773FD002851
:105A280006D16378002B02D00820FFF7ADFDF7BD43
:105A3800F6B23E80FBE7FF23019A0621200013718E
:105A48005371FFF7CFFC019B9871000AD871237836
:105A5800E8E78022D20097421BD1A2799A42E6D188
:105A6800E379B342E3D1FA23AAB29B009A42DED883
:105A7800654E34883580A4B2FFF744FD002854D120
:105A88000830FFF781FD614A338812689BB253637F
:105A9800CDE7A0212AB2C9008F4228D1A179994225
:105AA800C5D1E379B342C2D15948ABB21B185949A1
:105AB8009BB28B42BBD80A20574B584C5043268880
:105AC800198836B209B2FAF7B3FBABB200B2053B9C
:105AD80020800F2B00D8258023881BB2042BA6DD3D
:105AE80023881BB2142BA2DCFFF70CFD37E0C02281
:105AF800D20097421BD1A2799A4200D097E7E37966
:105B0800B34200D093E7424AABB29446414A634459
:105B18009BB2434E934200D989E73488358024B23A
:105B2800FFF7F0FC002800D17EE734807FE7E02211
:105B3800D200974218D1A2799A4200D077E7E37948
:105B4800B34200D073E7374B374A384C1A6000220B
:105B58002688374B2580B6B21A80FFF7DDFC00286F
:105B680000D161E7268062E78022120197421BD1AB
:105B7800A2799A4200D05AE7E379B34200D056E7B7
:105B8800ABB2032B00D952E72A4E3488358024B2B1
:105B9800FFF7B8FC0028C8D10830FFF7F5FC3088BB
:105BA80000B2FFF7BFFE42E7A022120197420ED1D2
:105BB800A2799A4200D03AE7E379B34200D036E7B7
:105BC8001D4BAAB29A4200D931E71C4EA5E7B02274
:105BD8001201974200D02AE7A2799A4200D026E71C
:105BE800E379B34200D022E7134BAAB29A4200D914
:105BF8001DE7134C0023E65E258075E7730500203A
:105C0800F3050020700500207403002050010020D7
:105C1800E40C0000C81900007A0300207203002079
:105C28007003002020000020D87700086E030020B1
:105C38006C0300206A030020DC050000240000201B
:105C48006603002010B50E4B0E491A7809888A425F
:105C58000ED10D49097808290AD15B78032B04D0A5
:105C6800062B04D1FFF7A8FE01E0FFF7AFFC10BD3B
:105C7800002AFCD1044A1278082AF8D15B78EFE7A9
:105C88007305002070050020F306002070B58026FB
:105C9800A0248025E405760131002D012000012291
:105CA800FDF714FC290001222000FDF70FFC042059
:105CB80000F098FB310000222000FDF707FC0420CB
:105CC80000F090FB290000222000FDF7FFFB70BDCB
:105CD80070B58026A0248025E405360131006D01C9
:105CE80020000022FDF7F2FB290000222000FDF72A
:105CF800EDFB042000F076FB310020000122FDF7C7
:105D0800E5FB290001222000FDF7E0FB042000F05C
:105D180069FB70BD8021A02070B501224901C00532
:105D2800FDF7D4FB012000F05DFB8021A0200122BB
:105D38000901C005FDF7CAFB8026012000F052FBCF
:105D480065257601A0203100C005FDF7B9FB041ECA
:105D580007D102008021A0200901C005FDF7B6FB8C
:105D680006E0013DEDB2002DECD1FFF7B1FF0124B3
:105D7800200070BD70B58025A0248026E4052D0183
:105D88002900760120000022FDF7A0FB3100002247
:105D98002000FDF79BFB022000F024FB29000122D4
:105DA8002000FDF793FB022000F01CFB29002000D7
:105DB8000022FDF78BFB310001222000FDF786FB56
:105DC80070BD70B58025A0248026E4052D0129002A
:105DD800760120000022FDF779FB31000122200026
:105DE800FDF774FB042000F0FDFA290001222000D1
:105DF800FDF76CFB042000F0F5FA290020000022D2
:105E0800FDF764FB310001222000FDF75FFB70BD48
:105E1800F8B580210400A0200022A02680270901CF
:105E2800C005FDF753FB0825F6053F0163B20122C3
:105E3800002B00DB0022802130004901FDF746FBE2
:105E4800022000F0CFFA012239003000FDF73EFBB6
:105E5800022000F0C7FA013D002239003000FDF7AA
:105E680035FB64000220EDB200F0BCFAE4B2002D6C
:105E7800DCD1F8BDF7B58027A026082500240190BD
:105E88003F01F605002239003000FDF71FFB022014
:105E980000F0A8FA390030000122FDF717FB802135
:105EA800640030004901E4B2FDF70AFB002801D084
:105EB8000134E4B2013D0120EDB200F093FA002D67
:105EC800E0D1019B002B03D1FFF77BFF2000FEBD33
:105ED800FFF750FFFAE70000F7B5FFF701FAB34BF9
:105EE8001A88B34B1A801A88002A03D01988B14A35
:105EF800914201D101221A80AF4B1A88AF4B1A8008
:105F08001A88002A03D01988AA4A914202D1AF22DE
:105F180092001A80AA4C1B8822689BB25363A94B33
:105F280000229A5EA84B1A801A88002A03D01A8881
:105F380012B2013201D10A221A80A44B00229A5EC1
:105F4800A34B1A801A88002A03D01A8812B2013289
:105F580001D100221A809F4B00229A5E9E4B1A8024
:105F68001A88002A03D01A8812B2013201D10022FD
:105F78001A80188800B2FFF7D5FC984B00229A5E69
:105F8800974B1A801A88002A03D01A8812B2013255
:105F980001D128221A80934B00229B5E5A1C92B290
:105FA800012A00D80023904A824913808C46002297
:105FB8008E488F4B8F4E03601F0019880837318039
:105FC800358819890097002D02D03588654501D19B
:105FD800002535804D1E884FADB2BD4200D9002145
:105FE80035888D4200D2C8E0002A00D00360200026
:105FF800FDF7D8FF00212000FEF7F0F97F4C2000C4
:10600800FEF7B2FA802220007D49FEF7A9FF7D4BFA
:10601800FA2201937C4B019918000093FCF72CFDA0
:10602800A02000222021C005FDF750FA32210020CF
:1060380000F082F9FA210120490000F07DF90320DF
:10604800724900F079F9FA210420890000F074F906
:106058000A21052000F070F90024002000F096F9CC
:10606800002809D00098FCF79BFDFFF74FF9FA22AA
:1060780001990098FCF700FD012000F087F900283D
:1060880009D00022624B63481A80FDF773FA012198
:106098006148FDF721FA022000F078F9002833D092
:1060A800A0200421C005FDF717FAE1230134A4B2AA
:1060B8005B019C4228D9338801339BB233803288F4
:1060C8003C4B9A4201D100233380544B1F78544BE8
:1060D8001878FBF789FC04000D001E2F5AD83800E9
:1060E800FBF782FC4F4A504BFBF7B6F922002B0016
:1060F800FAF7AAF9002804D04C4A138801339BB256
:106108001380FFF709FA0024032000F03FF9002864
:1061180002D00222464B1A70042000F037F90028FA
:106128000BD0022000F01EF9A02001220421C00596
:10613800FDF7CCF901223F4B1A70052000F026F933
:10614800002810D03C4D2800FFF756F86B79022B39
:1061580009D1286BFAF796F9314F3870686BFAF75E
:1061680091F92E4F3870354D2B78002B00D174E7FC
:10617800FFF768FD00232B706FE7314B009D9D42B0
:1061880003D02B000122318016E7002A00D12EE728
:106198002C4B2BE77842FBF727FC224A224BFBF7D4
:1061A8005BF90022284BFAF7C9FC9FE70078000842
:1061B80070050020FFFF000002780008740300202B
:1061C80050010020047800087203002006780008B7
:1061D80070030020087800086A0300200A78000885
:1061E800240000200C78000866030020200000200E
:1061F800007000086E030020FDFF0000540200201C
:10620800730600207C030020DC00002088130000B7
:1062180064030020400100200004005069030020AE
:1062280068030020CDCCCCCCCCCC06406C0300203D
:10623800270000202600002008030020F306002085
:10624800E0770008D877000800806640002370B522
:106258000C251C0012492800584301330A185460C1
:10626800946054704454062BF5D1FA210D4B8900E3
:106278001868F9F753FF802301385B0498420DD260
:10628800C021094A090650600848036A1B021B0A14
:106298000B43036207239460136070BDFEE7C0469A
:1062A800FC0600200000002010E000E000ED00E007
:1062B8001B4A70B51368002B07D01368013B1360A5
:1062C800002B02D10122174B1A7000220C2501263F
:1062D80015482C0054430319596800290AD05968F5
:1062E80001395960002905D15E70215C012901D16D
:1062F800996859600132062AEBD10C4B1A680132B1
:106308001A6019680A4A914201D100221A60094AA2
:1063180013780133DBB2092B00D90023137070BD49
:106328004807002044070020FC060020F80600204B
:10633800FFFFFF7FF4060020020010B5052800D9F2
:10634800FEE7012484F310880C205043044B1A18EC
:106358005160916000215170C45481F3108810BDC0
:10636800FC0600200300052800D9FEE7012282F37D
:1063780010880C2058430023034A11184B604B70B7
:10638800835483F310887047FC0600200200002025
:10639800052A09D80C214A43054B9B185978002235
:1063A800C8B2012901D15A7070471000FCE7C046F5
:1063B800FC06002000280FD0012800D1013001235D
:1063C80083F310880022054B1860054B1A7082F37E
:1063D80010881A78012AFCD17047C0464807002067
:1063E800440700200D4B70B50D4906001868F9F7F1
:1063F80095FE00230B4C46436568A168A26891424C
:10640800FCD006D95B189B1AB34200D370BD1100AB
:10641800F4E7A81AC318CB18F6E7C0460000002016
:1064280040420F0010E000E003008218934200D1C0
:10643800704719700133F9E770B500260C4C0D4D03
:10644800641BA410A64209D1002600F023F80A4CC8
:106458000A4D641BA410A64205D170BDB300EB58C9
:1064680098470136EEE7B300EB5898470136F2E754
:10647800546500085465000858650008546500080C
:10648800002310B59A4200D110BDCC5CC45401332E
:10649800F8E70000F8B5C046F8BC08BC9E4670474F
:1064A800F8B5C046F8BC08BC9E467047000000001E
:1064B80001B40248844601BC604700BF2D0000209B
:1064C80000000000000000000000000000000000C4
:1064D80001000000020000000300000004000000AA
:1064E80000000000000000000000000000000000A4
:1064F8000000000000000000000000000000000094
:106508000100000002000000030000000400000079
:106518000600000007000000080000000900000055
:1065280004020800010002000400060008000A0036
:106538000C00100020004000800000010804020444
:0C6548000801010101010103070100002E
:04655400E10000085A
:04655800B90000087E
:10655C000024F40001000000040000004443452D19
:10656C00323430332D56352E322E315F48414C00AB
:10657C0000700008280001010100000080220C4B73
:10658C0030B55C69D20222435A61EFF3108272B6C5
:10659C004C1CFF34401A0D68455004318C42FAD122
:1065AC008021490218690842FCD182F3108830BD61
:0465BC000020024079
:040000050800237557
:00000001FF
